:020000000D2AC7
:10000600831285128030F300F20108307202031861
:100016001C2873083505F1007108003A031D1528E0
:1000260085101628851485168512F30CF313F20A2B
:04003600082808008E
:10003A00831203137008F100F0010830FC00710804
:10004A00F40C03182C28FC0B2528F10100340310AA
:10005A003128F40C0318F107F10CF00CFC0B2E28D4
:02006A0008008C
:0C006C0083122B088A002A08820008007A
:10007800831205100B30B50003203408B5000320A7
:040088000514080053
:10008C0083120313F801F9011030FC00710DF80D07
:10009C00F90D7408F8027508031C750FF9020318A2
:1000AC005E287408F80775080318750FF907031014
:0A00BC00F00DF10DFC0B4C280800BC
:1000C60002308312FB008630FC009930FD00FD0BE8
:0C00D6006A28FC0B6A28FB0B6A28080053
:1000E20083120313FB01FA01F9018030F800F10CCD
:1000F200F00C031C85287408F90775080318750F9E
:10010200FA070318FB0A0310F01F8D287408FA0778
:1001120075080318750FFB07FB0CFA0CF90CF80CA9
:10012200031C78287B08F3007A08F2007908F100B2
:060132007808F00008004F
:0C01380007308312FD00FD0B9F2808001B
:0E01440083160511831212150C309504080065
:100152008312B001053030020318C52805100C3097
:10016200B5000320B5010320051463200330B40059
:100172003C2005100C30B50003200130B5000320EF
:0A01820005146320B00AAB28080042
:10018C0083161208013EF000F1010318F10A8312E4
:10019C003008F400F50171200630F2007008F4000C
:1001AC007108F50072080319E028F50CF40CF5132E
:1001BC00FF3ED9280430F1007408F00071080319CF
:1001CC00EB28F00D7010FF3EE52830307005F30081
:1001DC007408F0007508F100F10CF00CF113F10C3F
:1001EC00F00CF113700893000F309505730895040B
:0201FC000800F9
:1001FE00C33083129F05F0309F05F03083169F04A5
:10020E0083129F173008F000F00D7010F00D701073
:10021E0070089F041F149C209F149F1C1829000017
:10022E0014291F101E08F100F00183161E08F00499
:06023E000030F10408008D
:1002440036208A110A128000840AAA0A0319AB0A0A
:08025400F003031D222908003C
:0E025C008316051583121211F0309505080067
:10026A0083122208F0002308F100E830F40003307A
:10027A00F50071207008B0007108B1002408F00080
:10028A002508F1006430F4000030F5007120700890
:10029A003007A00031080318013E7107A1002808A1
:1002AA00F0000A30F4001D207008A0077108031836
:0E02BA00013EA1072908A0070318A10A0800A9
:1002C800831205100C30B50003200130B50003205F
:1002D800051405100930B50003200F30B5000320C0
:1002E800051405100A30B50003200F30B5000320AF
:1002F800051405100B30B50003200330B5000320AA
:10030800051405100F30B50003200130B500032097
:1003180005140630FB001330FC00AD30FD00FD0B6A
:100328009329FC0B9329FB0B93290000000005106F
:0E0338000F30B5000320B501032005140800A6
:10034600831205100430B5000320E830F4000330B2
:10035600F5003008F0003108F10046200A30F400BC
:100366000030F50046207808F0007908F1007008A2
:10037600B5000320051405100330B50003206430D2
:10038600F4000030F5003008F0003108F100462096
:100396000A30F4000030F50046207808F0007908AD
:1003A600F1007008B5000320051405100230B500F1
:1003B60003200A30F4000030F5003008F000310860
:1003C600F10046200A30F4000030F5004620780897
:1003D600F0007908F1007008B50003200514051037
:1003E6000130B50003200A30F4000030F500300873
:1003F600F0003108F10046207808F0007908F10095
:0A0406007008B5000320051408007B
:0A04100083129301151295120800E3
:10041A008312A001A101A201A301A401A501A601C1
:10042A00A701A801A9011830831685008312850146
:10043A0007309900083083169F0064212008B00015
:10044A002108B100A321AF0112109210C730831600
:10045A00920008227F30B000C6200330B000FF208F
:10046A007108013C031D3B2A7008903C03189C2A22
:10047A0003308312B000FF2002307102031D472AA5
:10048A00BC30700203189C2A83122708003A031D05
:10049A009C2AE830AC000330AD000330B000FF20E6
:1004AA007108013C031D5B2A7008903C03188B2AD3
:1004BA0003308312B000FF2002307102031D672A45
:1004CA00BC30700203188B2A0230FC004B30FD004E
:1004DA00FD0B6D2AFC0B6D2A01308312AC02031C42
:1004EA00AD0300302D06031D7C2A00302C06031DA7
:1004FA008A2A2108003C031D842A2008003C03188C
:10050A008A2A0130A700A6018B2A522A83122708B9
:10051A00031D9C2A2F08B4003C202F08AE00AF0A06
:10052A0004302F02031C9A2AAF010130A60083125D
:10053A000330B000FF2000307102031DA62A643088
:10054A0070020318E92A83122608013A031DE92AD0
:10055A006320D92AA90A2908093C0318B52AA9013E
:10056A00E92AA80A2808093C0318BC2AA801E92A8A
:10057A00A40A0319A50A2508003C031DC62A240853
:10058A00093C0318CA2AA401A501E92AA20A0319E7
:10059A00A30A2308003C031DD42A2208093C031895
:1005AA00D82AA201A301E92A2E08003A0319AF2A80
:1005BA002E08013A0319B62A2E08023A0319BD2A4F
:1005CA002E08033A0319CB2A8312270803191F2B73
:1005DA002108003C031DF32A2008003C03181F2BA6
:1005EA000130A002031CA1032008B0002108B100B9
:1005FA00A3210630FB001330FC00AD30FD00FD0BDB
:10060A00042BFC0B042BFB0B042B00000000003016
:10061A002106031D122B00302006031D1F2BA701E4
:10062A00A901A801A401A501A201A301AF01A22069
:10063A00A9202E212708031D282B35212008B000C8
:0A064A002108B100A321322A292B58
:02400E00E40FBD
:00000001FF
